:020000041000EA
:1000000098020020D5000010DD000010DF00001075
:1000100000000000000000000000000000000000E0
:10002000000000000000000000000000E1000010DF
:100030000000000000000000E3000010E5000010D8
:10004000E7000010E7000010E7000010E7000010D4
:10005000E7000010E7000010E7000010E7000010C4
:10006000E7000010E7000010E7000010E7000010B4
:1000700065100010D1100010E7000010E70000101C
:10008000E7000010E7000010E7000010E700001094
:10009000E7000010ED0E00104D0F0010E7000010FB
:1000A000E7000010E7000010000000000000000062
:1000B0000000000000000000000000000000000040
:1000C0000348854600F018FB00480047591400100B
:1000D000980200200448804704480047FEE7FEE7F6
:1000E000FEE7FEE7FEE7FEE7DD0E0010C1000010B0
:1000F00030B50B46014600202022012409E00D46C0
:10010000D5409D4205D31D469540491B2546954047
:1001100040191546521E002DF1DC30BD03460B433D
:100120009B0703D009E008C9121F08C0042AFAD2AD
:1001300003E00B780370401C491C521EF9D2704733
:10014000D2B201E00270401C491EFBD2704700226F
:10015000F6E710B513460A4604461946FFF7F0FFC6
:10016000204610BDF0B50C465C4085B0E40FE407B6
:1001700003944C000026640859009446490802463E
:100180000296224321D062460A431ED06200570DD8
:100190004A000E032303550D012402462C49240571
:1001A000781B1B0B360B40182343264361460090F7
:1001B0001C46501AB44103D30098401C009002E042
:1001C000921800985B41002803DA0020014605B030
:1001D000F0BD0020012109050746864611E064466E
:1001E0001D46141BB54106D36546521BB3417446E8
:1001F00007430C43A646CD074008490828439218F8
:100200005B4105460D43EAD11046184313D06046C2
:10021000194650407140084306D06046101AB34159
:1002200006D20122002306E000220123DB0702E0C0
:100230000122D2435310009874460105381C6141D5
:10024000029C039D0019694100F0B2F8BFE700006D
:10025000FD03000010B500229623114600F06FF850
:1002600010BD00000EB5C217C10F5040CA0740189C
:100270000021054B0293019200910A460B4600F0C3
:10028000A4F803B000BD0000330400000EB505491A
:100290000291002100910A460B46019100F095F869
:1002A00003B000BD33040000410040020122400AB7
:1002B000D205090E80187F2901DA0020704796299F
:1002C00003DC9622511AC84070479639884070471F
:1002D0004A0009030123090B1B051943094B10B5FB
:1002E000520D9A4201DA002010BD064B34339A4277
:1002F00003DC9A1A00F00AF810BD0349511888402F
:1003000010BD0000FF030000CDFBFFFF10B5202A49
:1003100004DB0846203AD040002110BD0B46D340F4
:10032000D0402024A21A91400843194610BD00294C
:1003300004DA401C490001D140084000704770B405
:100340000024050C05D11024000402D1002921D07D
:100350001124050E01D100020834050F01D100015E
:10036000241D850F01D18000A41C002801DB400062
:10037000641C002908D020252E1B0D46F540A14005
:1003800000D001212943084301061B1B000ADB1D85
:1003900002D5002070BC7047DB05181880180029B2
:1003A000F8DA401C4900F5D170BC400840007047A5
:1003B00010B5002B08DA0024401C614192185B4103
:1003C0001A4301D14008400010BDF0B51FB482B0FF
:1003D00005460C0003D0084600F071FF02E000F073
:1003E0006EFF2030024600902146284600F096F924
:1003F000049B059A04460F4618431143084314D042
:10040000184610431BD0009840210A1A1846059937
:10041000FFF77CFF05460E46009A0599049800F008
:100420007DF9084305D0012004E02046394607B095
:10043000F0BD0020C11705430E432C4337430099FC
:100440000E986305401A7905E40A00220C43FD0A60
:100450000A3002D500200146E9E70105101969417B
:100460000C9C0D9D00196941FFF7A2FFDFE700001A
:10047000F0B507460846584087B0C00F04904800C2
:100480000E46590040084908BC1A884105D2384632
:1004900031461E4617460B46024658004008104398
:1004A0004CD0300D039040055900400D490D05908A
:1004B000401A0290402872DA18030121000B090546
:1004C0000843019004980092002805D001995242F7
:1004D0000020884100920190029840210A1A019957
:1004E000009800F01BF905460C466B4607CB00F060
:1004F00025F9C0197141039A0E0D0023D7175640F4
:100500001A467A40164344D0049A002A2DD0029A03
:10051000012A039A15DC1205C01A914101263605FD
:10052000001C7141D20F059ED207009301920296E2
:100530002A462346FFF749FF07B0F0BD384631464B
:10054000FAE71605224A0F46B218C01AB741012130
:100550000905001C4F4100187F41114618187941C8
:10056000E20F10436D19644113E0E2076D08154373
:100570006408C2071443039A01261205C01A914168
:100580003605001C7141CE07400830434908C018A9
:1005900051412A462346FFF70BFFCDE7FFE70498BA
:1005A00001224000C117121A00238B4104983146E2
:1005B000C417381AA141EEE730B40124E4076340C0
:1005C00030BC55E730B40124E407614030BC4FE74C
:1005D0000000E0FFF0B51FB488B00B990998002423
:1005E00048400999C00F490049080991C0070B9973
:1005F0000090490049080B9109990898A6460843BC
:100600001CD00B990A98084318D00998012440007F
:10061000420D4800410D099824050003000B2043BA
:1006200009900B980003000B20430B9050181C49B5
:100630004018002201901446104605E000200146B3
:100640000DB0F0BD032801DA034600E003239C4609
:10065000C11A0AAE0AE05F0008ADED5B4F00F75B20
:100660007D430027AA187C41491C5B1E6145F2DDD1
:10067000410004AB5A522104120C0A43240C401CC2
:100680000828DFDB019802900099704601910090E4
:10069000059B049A07990698FFF797FED0E700009C
:1006A0000DFCFFFF70B54B005B0803430BD04B0004
:1006B0005C0D002633466542B341D417AD1AA34101
:1006C00002DB0020014670BD12053018514170BD9B
:1006D00010B5002904DB0124E40740428C41214687
:1006E000002B04DB1C460123DB075242A341994245
:1006F00000D1904210BD0000064C0125064E05E0D9
:10070000E36807CC2B430C3C98471034B442F7D332
:10071000FFF7DAFC90200010B020001010B5202A5E
:1007200004DB0146203A9140002010BD9140202377
:100730009C1A0346E3401943904010BD10B5202A8F
:1007400006DBCB170846203A1041C1170B4306E0E1
:100750000B461341D0402024A21A91400843194669
:1007600010BDFEB500231A461B1A8A4103DB002088
:10077000014603B0F0BD4A000D0301212D0B090510
:10078000520D0D43D10702D100186D41521E511078
:10079000FF31FF310131002704463E4638460097BD
:1007A00001910246012100200905FFF7AFFDC319A1
:1007B0007141F818324684468E464A4161462846C1
:1007C000611A904104D36046241A954176461F462B
:1007D000241900986D41401C00903428E1DDF9197E
:1007E00030467041091BA84103D20022D243134670
:1007F00001E00022134601980105381C7141FFF702
:10080000D7FDB6E710B51346002241608160002B8A
:1008100001D00824224301242243026010BD0000BD
:1008200010B5034800F008F80249086010BD000048
:100830002400002020000020F0B587B004460027E7
:100840005448006821780904084352490860207818
:1008500000281AD1084640686178090108434D49CB
:1008600048606178881CFFF7FDFC02460B46059145
:10087000049000200121890700F020FE0546FFF7C3
:1008800027FDC7B244494F4328E02078012803D10F
:10089000A77841494F4321E02078022801D18703FE
:1008A0001CE02078032801D1A78817E03948406868
:1008B000617809010843374948606178881CFFF76F
:1008C000D1FC02460B4605910490002001218907C6
:1008D00000F0F4FD0546FFF7FBFCC7B22D480068A9
:1008E000A17908432B49086000BF2A4800684007E7
:1008F000C00F0028F9D127480068217A090208436F
:100900002449086008460068E17909030843214941
:100910000860207A00281BDD217AC81EFFF7A2FCA0
:1009200005462A460B4600200121890700F0C6FD36
:10093000039102903846FFF7A9FC01910090039BB8
:10094000029AFFF70FFC05910490FFF7C1FC0746E0
:10095000E07900281BDDE179C81EFFF783FC05461E
:100960002A460B4600200121890700F0A7FD0391CC
:1009700002903846FFF78AFC01910090039B029A8F
:10098000FFF7F0FB05910490FFF7A2FC07463846FD
:1009900007B0F0BD0000024040420F0010B5044611
:1009A000002C04D00E2221460148FFF7B7FB10BDF2
:1009B0008400002010B50848007800280BD000F013
:1009C00011F806480068FFF76FFC84B2214604481E
:1009D00001F0E5FA00BF10BD5E00002068000020B5
:1009E00000C00040FEB54648007800287CD045484D
:1009F0000088401C434908804348407B002803D0BE
:100A000042480078002800D1FEBD4148847A7D210B
:100A1000C9004C43C57A4D43067B4E433D480078A0
:100A2000002804D001282BD0022864D138E03848AF
:100A3000807A7D21C900484332490988884215DB04
:100A4000334989882F4A1288514308462146FFF7C7
:100A50004FFB87B22E488088B84201DA2C4887883D
:100A60003846FFF7F7FB2C49086008E001202949C8
:100A7000087027498888FFF7EDFB274908603AE0AE
:100A8000601920490988884206D321498888FFF7E0
:100A9000E1FB2149086002E002201E4908702AE0BB
:100AA000601980191749098888421ED3601901907E
:100AB000144801880198081A009015498988009AFD
:100AC000514308463146FFF713FB11498988081A3C
:100AD00087B20F488088B84200DA00273846FFF70F
:100AE000B9FB0D49086005E007E000200A490860ED
:100AF0000849087000BF00BF00BF00BF84E70000C6
:100B00003100002032000020840000205E00002020
:100B1000500000206C0000206800002010B501F09B
:100B200003FA10BD00B500200649087006490860A8
:100B3000064908700649086006490860064801F041
:100B400023FA00BD5E000020680000206C00002039
:100B5000700000207400002000C0004010B500F0BC
:100B600003FA04462078002803D0FFF723FF002073
:100B700020706078002801D000206070E0780028A4
:100B800001D00020E0706079002801D00020607161
:100B9000A07900282DD0132000F02EF915480078F8
:100BA000401C14490870084600780A280CDC1248DA
:100BB000007800281BD101200F49087000200F4940
:100BC0000880FFF7ABFF12E00A48007814280BDC1E
:100BD0000948007801280AD1002007490870074910
:100BE0000880FFF79FFF02E0002002490870002004
:100BF000A07110BD30000020310000203200002024
:100C000010B502460F2A14DD1348806B1346103BC3
:100C10005C000323A34098430F4B98631846806BF6
:100C20001346103B5C000B46A34018430A4B9863E5
:100C30000FE00948406B54000323A3409843064B40
:100C400058631846406B54000B46A3401843024BB0
:100C50005863002010BD0000001002400146044807
:100C6000406801228A401040C840C0B2704700006E
:100C700000100240FFB504460D461E460B9F0021A2
:100C80002046FFF7BDFF012D10D1012F0ED14F4897
:100C900000690121A14088434C4908610846406928
:100CA0000121A1400843494948613BE0012D10D191
:100CB000002F0ED1454800690121A14088434349D6
:100CC0000861084640690121A14088433F494861C5
:100CD00028E0002D14D1012F12D13C484069012198
:100CE000A140884339494861084600690121A14073
:100CF000084336490861099848620298086311E080
:100D0000002D0FD1002F0DD1304800690121A140E5
:100D100088432E490861084640690121A140884363
:100D20002A494861022E0ED1284880690121A1403C
:100D30008843264988610846C1690120A040814353
:100D40002248C1611FE0002E0ED120488069012198
:100D5000A14008431D4988610846C0690121A1409E
:100D600088431A49C8610EE0012E0CD117488169E9
:100D70000120A040814315488161C0690121A14043
:100D800008431249C8611148816A0120A04081438B
:100D90000E488162806A0A99C907C90FA1400843B9
:100DA0000A4988620846C06A0121A1408843074970
:100DB000C8620846C06A0A998907C90FA14008435A
:100DC0000249C862002004B0F0BD000000100240DB
:100DD000012907D1074A5268012383401A43054B72
:100DE0005A6006E0034A5268012383409A43014B4C
:100DF0005A6070470010024000B503461846FFF7DE
:100E00002DFF012803D1184600F00AF807E0184624
:100E1000FFF724FF002802D1184600F00BF800BDB0
:100E200003494968012282409143014A5160704759
:100E30000010024003494968012282401143014ADF
:100E4000516070470010024000207047C206D20E69
:100E500001219140014A11607047000080E200E0EA
:100E6000C206D20E01219140014A11607047000074
:100E700080E200E0C206D20E01219140014A1160D9
:100E80007047000080E100E0C206D20E01219140CF
:100E9000014A11607047000080E100E0C206D20EF6
:100EA00001219140014A11607047000000E100E01B
:100EB000C206D20E01219140014A11607047000024
:100EC00000E100E001460448406901228A401043E5
:100ED000014A506100207047000002400148024969
:100EE0000860704700E1F5057C00002010B5012086
:100EF0000449C86004480068401C0349086000F0C9
:100F000045F810BD008000404400002070B5044644
:100F10000820FFF7D7FF1520FFF7B6FF1520FFF7D2
:100F20009FFF7D21C90007480068FFF7E1F8604393
:100F30000546012229460448FFF764FC1520FFF707
:100F4000B7FF70BD20000020008000400120044950
:100F5000C86004480068401C0249086070470000EF
:100F6000009000404C0000200048704734000020F2
:100F700010B507210348FFF7EAF808210248FFF7F8
:100F8000E6F810BD340000203C00002010B53348C6
:100F90000078401C3149087008464078401C487071
:100FA00008468078401C88700846C078401CC8708D
:100FB00008460079401C087108464079401C487179
:100FC0000846C088401CC88008460078012804DB19
:100FD000002008700120224908702048407802282B
:100FE00005DB00201D49487001201D4948701B4841
:100FF0008078062805DB00201849887001201849F0
:1010000088701648C0780A2805DB00201349C8708C
:1010100001201349C87011480079142805DB00200D
:101020000E49087101200E4908710C484079642866
:1010300005DB00200949487101200949487107482A
:10104000C0887D21C900884205DB00200349C88093
:10105000012003498871FFF781FD10BD3C0000208D
:101060003400002010B500240C20FFF7EFFE012013
:10107000800700F062F8032806D10120800740684D
:1010800004218843090748600120800700F055F8D3
:10109000022805D00120800700F04FF8062816D15D
:1010A000012080074068400840000121890748600E
:1010B00008460068C4B221460120800700F0EEF81F
:1010C000012080074068012108438907486010BD5E
:1010D00010B500240D20FFF7B9FE144800F02DF8DC
:1010E000032805D111484068042188430F4948600E
:1010F0000E4800F022F8022804D00C4800F01DF839
:10110000062812D109484068400840000749486055
:1011100008460068C4B22146044800F0BFF80348FE
:101120004068012108430149486010BD001000409B
:10113000014648698006C00F70470146886800076D
:10114000400F704770B504460D461348844206D1DF
:101150000D20FFF78FFE0D20FFF778FE09E001203C
:101160008007844205D10C20FFF784FE0C20FFF796
:101170006DFE60682978084360600748844203D1A7
:101180000D20FFF78BFE06E001208007844202D18C
:101190000C20FFF783FE70BD00100040F8B5044638
:1011A0000D460120800784420BD10020FFF78AFE04
:1011B00001210220FFF724FD01210320FFF720FD7C
:1011C0000DE0344884420AD10120FFF77BFE012163
:1011D0000C20FFF715FD01210D20FFF711FD606BBD
:1011E000C007C00F002801D1102700E00D272A48B2
:1011F00069680068FEF77CFF39460090FEF778FFCB
:10120000401E86B2F0B22062FF2000023040001281
:101210006062A068E968097889010843A060E8680D
:101220008078012803D1A06801210843A060E0680C
:1012300004218843E060E068297C89000843E0607D
:10124000E06880088000E060E068697C0843E06056
:10125000E06808218843E060E068297DC900084310
:10126000E060287D01280DD1E06830218843E060EE
:10127000E068E97C09010843E060E068A97C490175
:101280000843E060287A012803D12069202108431F
:101290002061F8BD001000402000002000B503468A
:1012A0000A4600BF1846FFF743FF0028FAD0114650
:1012B000184600F002F8104600BD0160704720217A
:1012C000020C01D010211046020A01D01046083944
:1012D000020901D01046091F820801D01046891E5C
:1012E000420801D0881E7047081A70474900CA0298
:1012F0000243100000D004204A0D01D00122104307
:10130000044A490D914201D102210843012800D12C
:1013100005207047FF070000F8B504464F1EC800BF
:101320000838211815461E46086849683A460623BB
:101330009A4310D02A463346FFF74CF93A46D2007A
:10134000083AA3181A687F1E5B68FFF791F8062217
:101350003B469343EED1022F23D0042F11D0062F0A
:101360002FD12A463346FFF735F9E36AA26AFFF721
:101370007FF82A463346FFF72DF9636A226AFFF7A2
:1013800077F82A463346FFF725F9E369A269FFF7A4
:101390006FF82A463346FFF71DF963692269FFF7A4
:1013A00067F82A463346FFF715F9E368A268FFF7A6
:1013B0005FF82A463346FFF70DF963682268FFF7A6
:1013C00057F8F8BD002210B5134610460149FEF744
:1013D000C9FE10BD0000F03F10B5FFF749F810BD81
:1013E000002210B5134610461146FEF7BBFE10BD95
:1013F00010B50721024A00200907FFF753F910BD75
:1014000001030000034A10B500201107FFF74AF955
:1014100010BD000001FDFFFF02E008C8121F08C157
:10142000002AFAD170477047002001E001C1121F65
:10143000002AFBD170470000014908607047000096
:10144000800000200248034948611020086170476D
:101450001377090000E000400EB5FFF7F5FCFFF739
:10146000DFF901200021009102230A460191029038
:101470001320FFF7FFFB00211320FFF7A9FC0B4906
:101480000B48FFF78BFE0B490948FFF75BFE0A4844
:10149000FFF784FAFFF76CFD0120FFF737FD00F03E
:1014A0002FFDFFF73BFB00BFFEE70000040000201C
:1014B000001000401C00002050000020F0B51FB4B8
:1014C00096B084460C460246199D18980390490030
:1014D00068006300490840080193002A01D00126F2
:1014E00000E000269E19FE4BF6185B109E422BD39F
:1014F0006E00039F0296002F00D00127F719F84EC7
:10150000F84BBE199E421FD3039E0346F64F33434A
:1015100009D03B469C4201D1002A04D0019B002AFD
:1015200005D0012604E0002039461BB0F0BD00269E
:101530009E19EE4B9E4207D8039F029E002F00D0BB
:101540000127F6199E4207D92B4660462146189A74
:10155000FFF742FF1BB0F0BD0023002C29DAE44E58
:10156000B04226DAE34EB04201DB022321E0DE4E38
:10157000B0421EDBE04E070DBE19142E09DD3427E4
:10158000BF1B039EFE400196BE40039FBE420BD090
:101590000FE0039F002F0CD11427BF1B0646FE400F
:1015A0000196BE40864204D1019BDE07F60F02235E
:1015B0009B1B0E46164318D1002D16DA002C03D0C3
:1015C000022B01D0012B06D00220FFF735FFFFF7D9
:1015D000F9FE1BB0F0BD0220FFF72EFFFFF7F2FE71
:1015E0000122D20751401BB0F0BD039E002E61D1F5
:1015F000BF4EB04220D1C148844201D1002A08D058
:10160000B948814209DB002D10DB189829461BB030
:10161000F0BD0020B4491BB0F0BD002D06DA012258
:101620002946D207189851401BB0F0BDB4497944FF
:10163000086849681BB0F0BDAB4FB84225D1002DFA
:101640001FDA002904D0B14212D1002A09D018E0D3
:10165000002A72D1A649E20F0020D20711431BB025
:10166000F0BD0020E20F0146D20711431BB0F0BDD0
:10167000B14206DA234600203946FEF773FD1BB05F
:10168000F0BD104621461BB0F0BDB14212DA012672
:10169000B607B54203D1234610461946FEE3994EDC
:1016A000B54207D1261E05DB1046314600F004FC8A
:1016B0001BB0F0BD67007F081646002A40D1002904
:1016C0000AD08B4A914229D1002C0EDD002D1CDB63
:1016D000002011461BB0F0BD022B16D0002C14D0F8
:1016E000012B12D1002C14DB0FE0002C28DA002D86
:1016F00009DB012B03D000207D491BB0F0BD002089
:1017000081491BB0F0BD012B03D0002001461BB066
:10171000F0BD00200121C9071BB0F0BD724A914203
:101720000ED1002C01DA002B17D0022B06D000209E
:10173000C043FEF797FD1BB0F0BD90E20120F8E733
:10174000E217521C94461A4307D000220892664CB6
:1017500062465B1E1A4307D009E00120FFF76CFECA
:10176000FFF73EFE1BB0F0BD0022644C0892674AB2
:1017700090427DDD664B674A98421FDD914202DC54
:10178000002D05DB4DE05848814217DB002D48DD78
:101790000220FFF751FEFFF72BFE05460E46002202
:1017A000534B21460898FEF715FF0846710049087B
:1017B000C00FC007014328461BB0F0BD914215DAA7
:1017C000002D2EDA0220FFF737FEFFF711FE054647
:1017D0000E460022464B21460898FEF7FBFE72009B
:1017E0005208C80FC0070243114617E03E4B99420A
:1017F00023DD002D15DD0220FFF71EFEFFF7F8FDAB
:1018000005460E4600223A4B21460898FEF7E2FEB6
:10181000084671004908C00FC007014328461BB0A5
:10182000F0BD0220FFF708FEFFF7ECFD4900490874
:10183000E20FD20711431BB0F0BD002230463946FB
:10184000FEF7BAFE012205460E46D243FEF72AFFF6
:10185000314A324BFEF7B6FE2A463346FEF7BAFE51
:101860000022284BFEF7AEFE07462A46334600E02C
:1018700064E0039110461946FEF7ACFE3A46039B1E
:10188000FEF7A8FE0746032209915207244B28467B
:101890003146FEF79FFE07910C90224A204B3846B6
:1018A0000999FEF797FE074601911F4A1F4B2846EC
:1018B0003146FEF78FFE3A46019BFEF77DFE074656
:1018C0000B460246099107990C98FEF7D1FD0025B9
:1018D0000E462846079B0C9AFEF76EFE3A4627E016
:1018E000FFFF1F00FFFF0F000000F03F0000E0FFC0
:1018F0000000F07F0000404301FCFFFF0000F0BF4C
:10190000560A00000000E03F0000F0FF0000E04148
:101910000000F043FFFFEF3F555555555555D53F56
:101920004715F73FFE822B6544DF5DF80BAE543E52
:10193000099BFEF747FE02460B4652E101250020B7
:101940002D05A94207DA352230463946FEF7AAFEB0
:1019500006463420C0430A151218FE48101803909A
:101960000803FD49000B01430F46FC49884201DC96
:10197000002003E0FA49884202DA0120119005E0D4
:10198000002011900398401C7F1B0390119805972D
:10199000C200F4480F9278448018436802683946C0
:1019A00030460D930292FEF707FE07910C903046E9
:1019B0000D9B029A0599FEF75BFD02460B4600203F
:1019C000E549FEF7CFFB09910490079B0C9AFEF7BF
:1019D00001FE129000201090E3480D467844006804
:1019E0000E90012178104907084311990D9B890435
:1019F00040180121C90447183946029A0E98FEF78B
:101A0000DBFD3246059BFEF7DDFD02460B4629460F
:101A10001098FEF7DFFD064602913B4629460E9AD6
:101A20001098FEF7D7FD079B0C9AFEF7CBFD3246C8
:101A3000029BFEF7C1FD099B049AFEF7CBFD0591C1
:101A4000129A0A902B4610461946FEF7C3FD064629
:101A50000246C6480F460B4606217844FFF75CFC59
:101A600032463B460091049010461946FEF7B2FDFF
:101A7000009B049AFEF7AEFD06460F462B4619461C
:101A8000129A1098FEF7F4FC059B0A9AFEF7A2FD45
:101A900032463B46FEF7ECFC109A079104902B4629
:101AA00010461946FEF796FDB14E002233460991C5
:101AB0000290FEF7DDFC079B049AFEF7D9FC00209C
:101AC0000746024633460091FEF776FD099B029ACF
:101AD000FEF772FD079B049AFEF774FD06460D9112
:101AE0003A462946009B1098FEF774FD07910C902A
:101AF0002B463046129A0D99FEF76CFD05460E46B0
:101B00003A46009B05990A98FEF764FD33462A463B
:101B1000FEF7AEFC02460B460746099107990C9862
:101B2000FEF7A6FC00250E462846079B0C9AFEF7FA
:101B300043FD3A46099BFEF745FD074607220991FA
:101B400052078C4B31462846FEF744FD0791009022
:101B5000894A884B38460999FEF73CFD07460191B2
:101B6000864A874B31462846FEF734FD3A46019BAC
:101B7000FEF77EFC834B7B440F9A9B181A685B68C8
:101B8000FEF776FC029009910398FEF76BFB059136
:101B90000490099B029A07990098FEF769FC7A4B1A
:101BA0007B440F9A9B181A685B6817460393FEF7ED
:101BB0005FFC059B049AFEF75BFC0E462846059BDE
:101BC000049AFEF7F9FC3A46039BFEF7F5FC079BE7
:101BD000009AFEF7F1FC099B029AFEF7F3FC02461D
:101BE0000B46199900200C900F461898FEF7F2FC4E
:101BF000029104903B460C9A19991898FEF7DCFC68
:101C00002A463346FEF7E6FC029B049AFEF730FCB8
:101C100009910E902A46334639460C98FEF7DAFCB5
:101C200006460F46099B0E9AFEF722FC574A0D46C0
:101C3000914220DB5242AA18024310D132463B4661
:101C4000FEF7BAFC04900391514A524B09990E9841
:101C5000FEF70EFC039B049AFEF73AFD1ED202200B
:101C6000FFF7EAFBFFF7C4FB49004908E20FD20780
:101C700011431BB0F0BD6A00474B52089A420DD386
:101C8000464AAA18024300D0CBE532463B46FEF74F
:101C900093FC099B0E9AFEF71BFDF5D96800002303
:101CA00040082C490393020D3D4B5218984223DD06
:101CB00001200005521CD04042195000400D401830
:101CC00038497944096813468C463749C1408B43EB
:101CD00012030121120B090551181422101AC140D8
:101CE0000391002D01DA484203906246304639469E
:101CF000FEF762FC06460F4632463B4609990E98AF
:101D0000FEF7B6FB00252A46284B28460591FEF72C
:101D100061FC07910C90264A264B28460599FEF750
:101D200059FC0091029032463B4628460599FEF741
:101D300043FC099B0E9AFEF745FC1F4A1F4BFEF71A
:101D400049FC009B029AFEF793FB07460B460246AE
:101D5000099135E001FCFFFF0000F03F8E98030081
:101D60007AB60B0066060000A8060000D205000047
:101D70000000084009C7EE3FFD033ADCF5015B14A3
:101D8000E02F3EBEA60400006C040000000090405E
:101D9000FE822B654715973C00CC904000346F3F86
:101DA0000000E03FC2030000FFFF0F00432EE63FAC
:101DB000396CA80C615C20BEEF39FAFE422EE63F7A
:101DC00007990C98FEF754FB05460E46079B0C9AA4
:101DD000FEF7F2FB3A46099BFEF7F4FB09912A460F
:101DE00033460E9010461946FEF7F4FB07460246AE
:101DF0002F480B46059105217844FFF78DFA3A46A6
:101E0000059BFEF7E7FB2A463346FEF7DBFB07465A
:101E1000019128463146099B0E9AFEF7DBFB099B90
:101E20000E9AFEF725FB012304910C9000229B07DC
:101E300038460199FEF7C0FB05910E903A462846B8
:101E40003146019BFEF7C6FB059B0E9AFEF78AF909
:101E5000049B0C9AFEF7B0FB2A463346FEF7ACFB18
:101E60000022144BFEF7AEFB064603980D46000514
:101E700041190915002912DC30462946039AFEF75C
:101E800011FCFFF733FA042801D1FFF7BBFA304603
:101E90002946039AFEF706FC064601E004E02918ED
:101EA0000B46324621460898FEF794FB1BB0F0BD66
:101EB000640200000000F03FF8B506460C46FEF74D
:101EC00050FC051E0F4600D00120014349000B487D
:101ED0004908411AC90F0DD0002E01D0012100E0A0
:101EE00000210C4361004908401AC00F02D10120B3
:101EF000FFF7A2FA28463946F8BD00000000F07F3F
:101F000010B50220054908600548406905490843A5
:101F100003494861FFF796FA10BD00000030024007
:101F2000000002400350000010B501200F49087066
:101F30000F48407B002809D000200E4908600E4958
:101F400008700E4908600E49086005E00849888855
:101F5000FEF780F90749086006480068FEF7A4F913
:101F600084B22146074800F023F810BD5E0000202F
:101F700084000020680000206C0000207000002019
:101F80007400002000C000400021C16300BF03E0D6
:101F9000C16100220262491C4029F9DB70470A46F0
:101FA000002102E0C1610262491C4029FADB70474E
:101FB00030B5024600230024642090602020906108
:101FC0009061642010615061502010600420D06343
:101FD000002002E0D0611162401C4028FADB192089
:101FE000C001506200209062D06201201063002086
:101FF0005063906301205060184630BD000000001F
:10200000000000000000F03F000000000000F83F6A
:1020100000000000000000000000004003B8E23FA4
:10202000000000000000000006D0CF43EBFD4C3E56
:10203000033333333333E33FFFAB6FDBB66DDB3F4B
:102040004D268F515555D53F01411DA96074D13F93
:1020500065DBC9934A86CD3FEF4E454A287ECA3F8D
:102060003E5555555555C53F93BDBE166CC166BF0F
:102070002CDE25AF6A56113FF16BD2C541BDBBBE08
:10208000D0A4BE726937663E000000000000000068
:10209000B020001000000020840000001814001080
:1020A00034210010840000201402000028140010C5
:1020B0000200010000000000B0AD010000000000BF
:1020C00000000020000300010000000005000000E7
:1020D00000000000000300000000000000000000FD
:1020E00000000000000000000000000000000000F0
:1020F00000000000000000000000000000000000E0
:102100006400E8038000640032000206020100005F
:1021100000000000000000000000000000000000BF
:10212000000000000000000000E1F50500E1F505F9
:0421300000000000AB
:04000005100000C126
:00000001FF
